
D:\STM32\Program\1.11_Odchudzanie\um0427\FWLib\project\RIDE\STM3210E-EVAL\stm32f10x_rcc.o:     file format elf32-littlearm
D:\STM32\Program\1.11_Odchudzanie\um0427\FWLib\project\RIDE\STM3210E-EVAL\stm32f10x_rcc.o

Disassembly of section .text.RCC_DeInit:

00000000 <RCC_DeInit>:
RCC_DeInit():
D:\STM32\Program\1.11_Odchudzanie\um0427\FWLib\library\src/stm32f10x_rcc.c:128
   0:	4a0d      	ldr	r2, [pc, #52]	(38 <RCC_DeInit+0x38>)
   2:	6813      	ldr	r3, [r2, #0]
   4:	f043 0301 	orr.w	r3, r3, #1	; 0x1
   8:	6013      	str	r3, [r2, #0]
D:\STM32\Program\1.11_Odchudzanie\um0427\FWLib\library\src/stm32f10x_rcc.c:131
   a:	6851      	ldr	r1, [r2, #4]
   c:	4b0b      	ldr	r3, [pc, #44]	(3c <RCC_DeInit+0x3c>)
   e:	ea01 0303 	and.w	r3, r1, r3
  12:	6053      	str	r3, [r2, #4]
D:\STM32\Program\1.11_Odchudzanie\um0427\FWLib\library\src/stm32f10x_rcc.c:134
  14:	6813      	ldr	r3, [r2, #0]
  16:	f023 7384 	bic.w	r3, r3, #17301504	; 0x1080000
  1a:	f423 3380 	bic.w	r3, r3, #65536	; 0x10000
  1e:	6013      	str	r3, [r2, #0]
D:\STM32\Program\1.11_Odchudzanie\um0427\FWLib\library\src/stm32f10x_rcc.c:137
  20:	6813      	ldr	r3, [r2, #0]
  22:	f423 2380 	bic.w	r3, r3, #262144	; 0x40000
  26:	6013      	str	r3, [r2, #0]
D:\STM32\Program\1.11_Odchudzanie\um0427\FWLib\library\src/stm32f10x_rcc.c:140
  28:	6853      	ldr	r3, [r2, #4]
  2a:	f423 03fe 	bic.w	r3, r3, #8323072	; 0x7f0000
  2e:	6053      	str	r3, [r2, #4]
D:\STM32\Program\1.11_Odchudzanie\um0427\FWLib\library\src/stm32f10x_rcc.c:143
  30:	2300      	movs	r3, #0
  32:	6093      	str	r3, [r2, #8]
D:\STM32\Program\1.11_Odchudzanie\um0427\FWLib\library\src/stm32f10x_rcc.c:144
  34:	4770      	bx	lr
  36:	46c0      	nop			(mov r8, r8)
  38:	40021000 	.word	0x40021000
  3c:	f8ff0000 	.word	0xf8ff0000
Disassembly of section .text.RCC_HSEConfig:

00000000 <RCC_HSEConfig>:
RCC_HSEConfig():
D:\STM32\Program\1.11_Odchudzanie\um0427\FWLib\library\src/stm32f10x_rcc.c:167
   0:	4a0c      	ldr	r2, [pc, #48]	(34 <RCC_HSEConfig+0x34>)
D:\STM32\Program\1.11_Odchudzanie\um0427\FWLib\library\src/stm32f10x_rcc.c:173
   2:	f5b0 3f80 	cmp.w	r0, #65536	; 0x10000
D:\STM32\Program\1.11_Odchudzanie\um0427\FWLib\library\src/stm32f10x_rcc.c:167
   6:	6813      	ldr	r3, [r2, #0]
   8:	f423 3380 	bic.w	r3, r3, #65536	; 0x10000
   c:	6013      	str	r3, [r2, #0]
D:\STM32\Program\1.11_Odchudzanie\um0427\FWLib\library\src/stm32f10x_rcc.c:170
   e:	6813      	ldr	r3, [r2, #0]
  10:	f423 2380 	bic.w	r3, r3, #262144	; 0x40000
  14:	6013      	str	r3, [r2, #0]
D:\STM32\Program\1.11_Odchudzanie\um0427\FWLib\library\src/stm32f10x_rcc.c:173
  16:	d003      	beq.n	20 <RCC_HSEConfig+0x20>
  18:	f5b0 2f80 	cmp.w	r0, #262144	; 0x40000
  1c:	d004      	beq.n	28 <RCC_HSEConfig+0x28>
  1e:	e007      	b.n	30 <RCC_HSEConfig+0x30>
D:\STM32\Program\1.11_Odchudzanie\um0427\FWLib\library\src/stm32f10x_rcc.c:177
  20:	6813      	ldr	r3, [r2, #0]
  22:	f443 3380 	orr.w	r3, r3, #65536	; 0x10000
  26:	e002      	b.n	2e <RCC_HSEConfig+0x2e>
D:\STM32\Program\1.11_Odchudzanie\um0427\FWLib\library\src/stm32f10x_rcc.c:182
  28:	6813      	ldr	r3, [r2, #0]
  2a:	f443 23a0 	orr.w	r3, r3, #327680	; 0x50000
  2e:	6013      	str	r3, [r2, #0]
D:\STM32\Program\1.11_Odchudzanie\um0427\FWLib\library\src/stm32f10x_rcc.c:188
  30:	4770      	bx	lr
  32:	46c0      	nop			(mov r8, r8)
  34:	40021000 	.word	0x40021000
Disassembly of section .text.RCC_AdjustHSICalibrationValue:

00000000 <RCC_AdjustHSICalibrationValue>:
RCC_AdjustHSICalibrationValue():
D:\STM32\Program\1.11_Odchudzanie\um0427\FWLib\library\src/stm32f10x_rcc.c:239
   0:	4a03      	ldr	r2, [pc, #12]	(10 <RCC_AdjustHSICalibrationValue+0x10>)
   2:	6813      	ldr	r3, [r2, #0]
D:\STM32\Program\1.11_Odchudzanie\um0427\FWLib\library\src/stm32f10x_rcc.c:242
   4:	f023 03f8 	bic.w	r3, r3, #248	; 0xf8
D:\STM32\Program\1.11_Odchudzanie\um0427\FWLib\library\src/stm32f10x_rcc.c:245
   8:	ea43 03c0 	orr.w	r3, r3, r0, lsl #3
D:\STM32\Program\1.11_Odchudzanie\um0427\FWLib\library\src/stm32f10x_rcc.c:248
   c:	6013      	str	r3, [r2, #0]
D:\STM32\Program\1.11_Odchudzanie\um0427\FWLib\library\src/stm32f10x_rcc.c:249
   e:	4770      	bx	lr
  10:	40021000 	.word	0x40021000
Disassembly of section .text.RCC_HSICmd:

00000000 <RCC_HSICmd>:
RCC_HSICmd():
D:\STM32\Program\1.11_Odchudzanie\um0427\FWLib\library\src/stm32f10x_rcc.c:266
   0:	4b01      	ldr	r3, [pc, #4]	(8 <RCC_HSICmd+0x8>)
   2:	6018      	str	r0, [r3, #0]
D:\STM32\Program\1.11_Odchudzanie\um0427\FWLib\library\src/stm32f10x_rcc.c:267
   4:	4770      	bx	lr
   6:	46c0      	nop			(mov r8, r8)
   8:	42420000 	.word	0x42420000
Disassembly of section .text.RCC_PLLConfig:

00000000 <RCC_PLLConfig>:
RCC_PLLConfig():
D:\STM32\Program\1.11_Odchudzanie\um0427\FWLib\library\src/stm32f10x_rcc.c:294
   0:	4b03      	ldr	r3, [pc, #12]	(10 <RCC_PLLConfig+0x10>)
   2:	685a      	ldr	r2, [r3, #4]
D:\STM32\Program\1.11_Odchudzanie\um0427\FWLib\library\src/stm32f10x_rcc.c:300
   4:	f422 127c 	bic.w	r2, r2, #4128768	; 0x3f0000
   8:	4310      	orrs	r0, r2
   a:	4308      	orrs	r0, r1
D:\STM32\Program\1.11_Odchudzanie\um0427\FWLib\library\src/stm32f10x_rcc.c:303
   c:	6058      	str	r0, [r3, #4]
D:\STM32\Program\1.11_Odchudzanie\um0427\FWLib\library\src/stm32f10x_rcc.c:304
   e:	4770      	bx	lr
  10:	40021000 	.word	0x40021000
Disassembly of section .text.RCC_PLLCmd:

00000000 <RCC_PLLCmd>:
RCC_PLLCmd():
D:\STM32\Program\1.11_Odchudzanie\um0427\FWLib\library\src/stm32f10x_rcc.c:320
   0:	4b01      	ldr	r3, [pc, #4]	(8 <RCC_PLLCmd+0x8>)
   2:	6018      	str	r0, [r3, #0]
D:\STM32\Program\1.11_Odchudzanie\um0427\FWLib\library\src/stm32f10x_rcc.c:321
   4:	4770      	bx	lr
   6:	46c0      	nop			(mov r8, r8)
   8:	42420060 	.word	0x42420060
Disassembly of section .text.RCC_SYSCLKConfig:

00000000 <RCC_SYSCLKConfig>:
RCC_SYSCLKConfig():
D:\STM32\Program\1.11_Odchudzanie\um0427\FWLib\library\src/stm32f10x_rcc.c:341
   0:	4b03      	ldr	r3, [pc, #12]	(10 <RCC_SYSCLKConfig+0x10>)
   2:	685a      	ldr	r2, [r3, #4]
D:\STM32\Program\1.11_Odchudzanie\um0427\FWLib\library\src/stm32f10x_rcc.c:344
   4:	f022 0203 	bic.w	r2, r2, #3	; 0x3
D:\STM32\Program\1.11_Odchudzanie\um0427\FWLib\library\src/stm32f10x_rcc.c:347
   8:	4310      	orrs	r0, r2
D:\STM32\Program\1.11_Odchudzanie\um0427\FWLib\library\src/stm32f10x_rcc.c:350
   a:	6058      	str	r0, [r3, #4]
D:\STM32\Program\1.11_Odchudzanie\um0427\FWLib\library\src/stm32f10x_rcc.c:351
   c:	4770      	bx	lr
   e:	46c0      	nop			(mov r8, r8)
  10:	40021000 	.word	0x40021000
Disassembly of section .text.RCC_GetSYSCLKSource:

00000000 <RCC_GetSYSCLKSource>:
RCC_GetSYSCLKSource():
D:\STM32\Program\1.11_Odchudzanie\um0427\FWLib\library\src/stm32f10x_rcc.c:366
   0:	4b02      	ldr	r3, [pc, #8]	(c <RCC_GetSYSCLKSource+0xc>)
   2:	6858      	ldr	r0, [r3, #4]
D:\STM32\Program\1.11_Odchudzanie\um0427\FWLib\library\src/stm32f10x_rcc.c:367
   4:	f000 000c 	and.w	r0, r0, #12	; 0xc
   8:	4770      	bx	lr
   a:	46c0      	nop			(mov r8, r8)
   c:	40021000 	.word	0x40021000
Disassembly of section .text.RCC_HCLKConfig:

00000000 <RCC_HCLKConfig>:
RCC_HCLKConfig():
D:\STM32\Program\1.11_Odchudzanie\um0427\FWLib\library\src/stm32f10x_rcc.c:394
   0:	4b03      	ldr	r3, [pc, #12]	(10 <RCC_HCLKConfig+0x10>)
   2:	685a      	ldr	r2, [r3, #4]
D:\STM32\Program\1.11_Odchudzanie\um0427\FWLib\library\src/stm32f10x_rcc.c:397
   4:	f022 02f0 	bic.w	r2, r2, #240	; 0xf0
D:\STM32\Program\1.11_Odchudzanie\um0427\FWLib\library\src/stm32f10x_rcc.c:400
   8:	4310      	orrs	r0, r2
D:\STM32\Program\1.11_Odchudzanie\um0427\FWLib\library\src/stm32f10x_rcc.c:403
   a:	6058      	str	r0, [r3, #4]
D:\STM32\Program\1.11_Odchudzanie\um0427\FWLib\library\src/stm32f10x_rcc.c:404
   c:	4770      	bx	lr
   e:	46c0      	nop			(mov r8, r8)
  10:	40021000 	.word	0x40021000
Disassembly of section .text.RCC_PCLK1Config:

00000000 <RCC_PCLK1Config>:
RCC_PCLK1Config():
D:\STM32\Program\1.11_Odchudzanie\um0427\FWLib\library\src/stm32f10x_rcc.c:427
   0:	4b03      	ldr	r3, [pc, #12]	(10 <RCC_PCLK1Config+0x10>)
   2:	685a      	ldr	r2, [r3, #4]
D:\STM32\Program\1.11_Odchudzanie\um0427\FWLib\library\src/stm32f10x_rcc.c:430
   4:	f422 62e0 	bic.w	r2, r2, #1792	; 0x700
D:\STM32\Program\1.11_Odchudzanie\um0427\FWLib\library\src/stm32f10x_rcc.c:433
   8:	4310      	orrs	r0, r2
D:\STM32\Program\1.11_Odchudzanie\um0427\FWLib\library\src/stm32f10x_rcc.c:436
   a:	6058      	str	r0, [r3, #4]
D:\STM32\Program\1.11_Odchudzanie\um0427\FWLib\library\src/stm32f10x_rcc.c:437
   c:	4770      	bx	lr
   e:	46c0      	nop			(mov r8, r8)
  10:	40021000 	.word	0x40021000
Disassembly of section .text.RCC_PCLK2Config:

00000000 <RCC_PCLK2Config>:
RCC_PCLK2Config():
D:\STM32\Program\1.11_Odchudzanie\um0427\FWLib\library\src/stm32f10x_rcc.c:460
   0:	4a03      	ldr	r2, [pc, #12]	(10 <RCC_PCLK2Config+0x10>)
   2:	6853      	ldr	r3, [r2, #4]
D:\STM32\Program\1.11_Odchudzanie\um0427\FWLib\library\src/stm32f10x_rcc.c:463
   4:	f423 5360 	bic.w	r3, r3, #14336	; 0x3800
D:\STM32\Program\1.11_Odchudzanie\um0427\FWLib\library\src/stm32f10x_rcc.c:466
   8:	ea43 03c0 	orr.w	r3, r3, r0, lsl #3
D:\STM32\Program\1.11_Odchudzanie\um0427\FWLib\library\src/stm32f10x_rcc.c:469
   c:	6053      	str	r3, [r2, #4]
D:\STM32\Program\1.11_Odchudzanie\um0427\FWLib\library\src/stm32f10x_rcc.c:470
   e:	4770      	bx	lr
  10:	40021000 	.word	0x40021000
Disassembly of section .text.RCC_ITConfig:

00000000 <RCC_ITConfig>:
RCC_ITConfig():
D:\STM32\Program\1.11_Odchudzanie\um0427\FWLib\library\src/stm32f10x_rcc.c:494
   0:	b121      	cbz	r1, c <RCC_ITConfig+0xc>
D:\STM32\Program\1.11_Odchudzanie\um0427\FWLib\library\src/stm32f10x_rcc.c:497
   2:	4a05      	ldr	r2, [pc, #20]	(18 <RCC_ITConfig+0x18>)
   4:	7813      	ldrb	r3, [r2, #0]
   6:	ea40 0303 	orr.w	r3, r0, r3
   a:	e003      	b.n	14 <RCC_ITConfig+0x14>
D:\STM32\Program\1.11_Odchudzanie\um0427\FWLib\library\src/stm32f10x_rcc.c:502
   c:	4a02      	ldr	r2, [pc, #8]	(18 <RCC_ITConfig+0x18>)
   e:	7813      	ldrb	r3, [r2, #0]
  10:	ea23 0300 	bic.w	r3, r3, r0
  14:	7013      	strb	r3, [r2, #0]
D:\STM32\Program\1.11_Odchudzanie\um0427\FWLib\library\src/stm32f10x_rcc.c:504
  16:	4770      	bx	lr
  18:	40021009 	.word	0x40021009
Disassembly of section .text.RCC_USBCLKConfig:

00000000 <RCC_USBCLKConfig>:
RCC_USBCLKConfig():
D:\STM32\Program\1.11_Odchudzanie\um0427\FWLib\library\src/stm32f10x_rcc.c:524
   0:	4b01      	ldr	r3, [pc, #4]	(8 <RCC_USBCLKConfig+0x8>)
   2:	6018      	str	r0, [r3, #0]
D:\STM32\Program\1.11_Odchudzanie\um0427\FWLib\library\src/stm32f10x_rcc.c:525
   4:	4770      	bx	lr
   6:	46c0      	nop			(mov r8, r8)
   8:	424200d8 	.word	0x424200d8
Disassembly of section .text.RCC_ADCCLKConfig:

00000000 <RCC_ADCCLKConfig>:
RCC_ADCCLKConfig():
D:\STM32\Program\1.11_Odchudzanie\um0427\FWLib\library\src/stm32f10x_rcc.c:547
   0:	4b03      	ldr	r3, [pc, #12]	(10 <RCC_ADCCLKConfig+0x10>)
   2:	685a      	ldr	r2, [r3, #4]
D:\STM32\Program\1.11_Odchudzanie\um0427\FWLib\library\src/stm32f10x_rcc.c:550
   4:	f422 4240 	bic.w	r2, r2, #49152	; 0xc000
D:\STM32\Program\1.11_Odchudzanie\um0427\FWLib\library\src/stm32f10x_rcc.c:553
   8:	4310      	orrs	r0, r2
D:\STM32\Program\1.11_Odchudzanie\um0427\FWLib\library\src/stm32f10x_rcc.c:556
   a:	6058      	str	r0, [r3, #4]
D:\STM32\Program\1.11_Odchudzanie\um0427\FWLib\library\src/stm32f10x_rcc.c:557
   c:	4770      	bx	lr
   e:	46c0      	nop			(mov r8, r8)
  10:	40021000 	.word	0x40021000
Disassembly of section .text.RCC_LSEConfig:

00000000 <RCC_LSEConfig>:
RCC_LSEConfig():
D:\STM32\Program\1.11_Odchudzanie\um0427\FWLib\library\src/stm32f10x_rcc.c:578
   0:	4a06      	ldr	r2, [pc, #24]	(1c <RCC_LSEConfig+0x1c>)
   2:	2300      	movs	r3, #0
D:\STM32\Program\1.11_Odchudzanie\um0427\FWLib\library\src/stm32f10x_rcc.c:584
   4:	2801      	cmp	r0, #1
D:\STM32\Program\1.11_Odchudzanie\um0427\FWLib\library\src/stm32f10x_rcc.c:578
   6:	7013      	strb	r3, [r2, #0]
D:\STM32\Program\1.11_Odchudzanie\um0427\FWLib\library\src/stm32f10x_rcc.c:581
   8:	7013      	strb	r3, [r2, #0]
D:\STM32\Program\1.11_Odchudzanie\um0427\FWLib\library\src/stm32f10x_rcc.c:584
   a:	d002      	beq.n	12 <RCC_LSEConfig+0x12>
   c:	2804      	cmp	r0, #4
   e:	d002      	beq.n	16 <RCC_LSEConfig+0x16>
  10:	e003      	b.n	1a <RCC_LSEConfig+0x1a>
D:\STM32\Program\1.11_Odchudzanie\um0427\FWLib\library\src/stm32f10x_rcc.c:588
  12:	7010      	strb	r0, [r2, #0]
D:\STM32\Program\1.11_Odchudzanie\um0427\FWLib\library\src/stm32f10x_rcc.c:589
  14:	e001      	b.n	1a <RCC_LSEConfig+0x1a>
D:\STM32\Program\1.11_Odchudzanie\um0427\FWLib\library\src/stm32f10x_rcc.c:593
  16:	2305      	movs	r3, #5
  18:	7013      	strb	r3, [r2, #0]
D:\STM32\Program\1.11_Odchudzanie\um0427\FWLib\library\src/stm32f10x_rcc.c:599
  1a:	4770      	bx	lr
  1c:	40021020 	.word	0x40021020
Disassembly of section .text.RCC_LSICmd:

00000000 <RCC_LSICmd>:
RCC_LSICmd():
D:\STM32\Program\1.11_Odchudzanie\um0427\FWLib\library\src/stm32f10x_rcc.c:615
   0:	4b01      	ldr	r3, [pc, #4]	(8 <RCC_LSICmd+0x8>)
   2:	6018      	str	r0, [r3, #0]
D:\STM32\Program\1.11_Odchudzanie\um0427\FWLib\library\src/stm32f10x_rcc.c:616
   4:	4770      	bx	lr
   6:	46c0      	nop			(mov r8, r8)
   8:	42420480 	.word	0x42420480
Disassembly of section .text.RCC_RTCCLKConfig:

00000000 <RCC_RTCCLKConfig>:
RCC_RTCCLKConfig():
D:\STM32\Program\1.11_Odchudzanie\um0427\FWLib\library\src/stm32f10x_rcc.c:638
   0:	4b02      	ldr	r3, [pc, #8]	(c <RCC_RTCCLKConfig+0xc>)
   2:	6a1a      	ldr	r2, [r3, #32]
   4:	4310      	orrs	r0, r2
   6:	6218      	str	r0, [r3, #32]
D:\STM32\Program\1.11_Odchudzanie\um0427\FWLib\library\src/stm32f10x_rcc.c:639
   8:	4770      	bx	lr
   a:	46c0      	nop			(mov r8, r8)
   c:	40021000 	.word	0x40021000
Disassembly of section .text.RCC_RTCCLKCmd:

00000000 <RCC_RTCCLKCmd>:
RCC_RTCCLKCmd():
D:\STM32\Program\1.11_Odchudzanie\um0427\FWLib\library\src/stm32f10x_rcc.c:656
   0:	4b01      	ldr	r3, [pc, #4]	(8 <RCC_RTCCLKCmd+0x8>)
   2:	6018      	str	r0, [r3, #0]
D:\STM32\Program\1.11_Odchudzanie\um0427\FWLib\library\src/stm32f10x_rcc.c:657
   4:	4770      	bx	lr
   6:	46c0      	nop			(mov r8, r8)
   8:	4242043c 	.word	0x4242043c
Disassembly of section .text.RCC_GetClocksFreq:

00000000 <RCC_GetClocksFreq>:
RCC_GetClocksFreq():
D:\STM32\Program\1.11_Odchudzanie\um0427\FWLib\library\src/stm32f10x_rcc.c:672
   0:	491e      	ldr	r1, [pc, #120]	(7c <RCC_GetClocksFreq+0x7c>)
D:\STM32\Program\1.11_Odchudzanie\um0427\FWLib\library\src/stm32f10x_rcc.c:668
   2:	b510      	push	{r4, lr}
D:\STM32\Program\1.11_Odchudzanie\um0427\FWLib\library\src/stm32f10x_rcc.c:672
   4:	684b      	ldr	r3, [r1, #4]
D:\STM32\Program\1.11_Odchudzanie\um0427\FWLib\library\src/stm32f10x_rcc.c:668
   6:	4604      	mov	r4, r0
D:\STM32\Program\1.11_Odchudzanie\um0427\FWLib\library\src/stm32f10x_rcc.c:674
   8:	f003 030c 	and.w	r3, r3, #12	; 0xc
   c:	2b04      	cmp	r3, #4
   e:	d013      	beq.n	38 <RCC_GetClocksFreq+0x38>
  10:	2b08      	cmp	r3, #8
  12:	d111      	bne.n	38 <RCC_GetClocksFreq+0x38>
D:\STM32\Program\1.11_Odchudzanie\um0427\FWLib\library\src/stm32f10x_rcc.c:686
  14:	684b      	ldr	r3, [r1, #4]
D:\STM32\Program\1.11_Odchudzanie\um0427\FWLib\library\src/stm32f10x_rcc.c:687
  16:	f3c3 4383 	ubfx	r3, r3, #18, #4
  1a:	1c9a      	adds	r2, r3, #2
D:\STM32\Program\1.11_Odchudzanie\um0427\FWLib\library\src/stm32f10x_rcc.c:689
  1c:	684b      	ldr	r3, [r1, #4]
D:\STM32\Program\1.11_Odchudzanie\um0427\FWLib\library\src/stm32f10x_rcc.c:691
  1e:	f413 3f80 	tst.w	r3, #65536	; 0x10000
  22:	d003      	beq.n	2c <RCC_GetClocksFreq+0x2c>
D:\STM32\Program\1.11_Odchudzanie\um0427\FWLib\library\src/stm32f10x_rcc.c:698
  24:	684b      	ldr	r3, [r1, #4]
  26:	f413 3f00 	tst.w	r3, #131072	; 0x20000
  2a:	d001      	beq.n	30 <RCC_GetClocksFreq+0x30>
D:\STM32\Program\1.11_Odchudzanie\um0427\FWLib\library\src/stm32f10x_rcc.c:701
  2c:	4b14      	ldr	r3, [pc, #80]	(80 <RCC_GetClocksFreq+0x80>)
  2e:	e000      	b.n	32 <RCC_GetClocksFreq+0x32>
D:\STM32\Program\1.11_Odchudzanie\um0427\FWLib\library\src/stm32f10x_rcc.c:705
  30:	4b14      	ldr	r3, [pc, #80]	(84 <RCC_GetClocksFreq+0x84>)
  32:	fb02 f303 	mul.w	r3, r2, r3
  36:	e000      	b.n	3a <RCC_GetClocksFreq+0x3a>
D:\STM32\Program\1.11_Odchudzanie\um0427\FWLib\library\src/stm32f10x_rcc.c:711
  38:	4b12      	ldr	r3, [pc, #72]	(84 <RCC_GetClocksFreq+0x84>)
D:\STM32\Program\1.11_Odchudzanie\um0427\FWLib\library\src/stm32f10x_rcc.c:717
  3a:	4910      	ldr	r1, [pc, #64]	(7c <RCC_GetClocksFreq+0x7c>)
D:\STM32\Program\1.11_Odchudzanie\um0427\FWLib\library\src/stm32f10x_rcc.c:711
  3c:	6023      	str	r3, [r4, #0]
D:\STM32\Program\1.11_Odchudzanie\um0427\FWLib\library\src/stm32f10x_rcc.c:717
  3e:	684b      	ldr	r3, [r1, #4]
D:\STM32\Program\1.11_Odchudzanie\um0427\FWLib\library\src/stm32f10x_rcc.c:722
  40:	4811      	ldr	r0, [pc, #68]	(88 <RCC_GetClocksFreq+0x88>)
  42:	f3c3 1303 	ubfx	r3, r3, #4, #4
  46:	5cc3      	ldrb	r3, [r0, r3]
  48:	6822      	ldr	r2, [r4, #0]
  4a:	40da      	lsrs	r2, r3
  4c:	6062      	str	r2, [r4, #4]
D:\STM32\Program\1.11_Odchudzanie\um0427\FWLib\library\src/stm32f10x_rcc.c:725
  4e:	684b      	ldr	r3, [r1, #4]
D:\STM32\Program\1.11_Odchudzanie\um0427\FWLib\library\src/stm32f10x_rcc.c:730
  50:	f3c3 2302 	ubfx	r3, r3, #8, #3
  54:	5cc3      	ldrb	r3, [r0, r3]
  56:	fa32 f303 	lsrs.w	r3, r2, r3
  5a:	60a3      	str	r3, [r4, #8]
D:\STM32\Program\1.11_Odchudzanie\um0427\FWLib\library\src/stm32f10x_rcc.c:733
  5c:	684b      	ldr	r3, [r1, #4]
D:\STM32\Program\1.11_Odchudzanie\um0427\FWLib\library\src/stm32f10x_rcc.c:738
  5e:	f3c3 23c2 	ubfx	r3, r3, #11, #3
  62:	5cc3      	ldrb	r3, [r0, r3]
  64:	40da      	lsrs	r2, r3
  66:	60e2      	str	r2, [r4, #12]
D:\STM32\Program\1.11_Odchudzanie\um0427\FWLib\library\src/stm32f10x_rcc.c:741
  68:	684b      	ldr	r3, [r1, #4]
D:\STM32\Program\1.11_Odchudzanie\um0427\FWLib\library\src/stm32f10x_rcc.c:746
  6a:	f3c3 3381 	ubfx	r3, r3, #14, #2
  6e:	181b      	adds	r3, r3, r0
  70:	7c1b      	ldrb	r3, [r3, #16]
  72:	fbb2 f2f3 	udiv	r2, r2, r3
  76:	6122      	str	r2, [r4, #16]
D:\STM32\Program\1.11_Odchudzanie\um0427\FWLib\library\src/stm32f10x_rcc.c:747
  78:	bd10      	pop	{r4, pc}
  7a:	46c0      	nop			(mov r8, r8)
  7c:	40021000 	.word	0x40021000
  80:	003d0900 	.word	0x003d0900
  84:	007a1200 	.word	0x007a1200
  88:	00000000 	.word	0x00000000
Disassembly of section .text.RCC_AHBPeriphClockCmd:

00000000 <RCC_AHBPeriphClockCmd>:
RCC_AHBPeriphClockCmd():
D:\STM32\Program\1.11_Odchudzanie\um0427\FWLib\library\src/stm32f10x_rcc.c:773
   0:	b121      	cbz	r1, c <RCC_AHBPeriphClockCmd+0xc>
D:\STM32\Program\1.11_Odchudzanie\um0427\FWLib\library\src/stm32f10x_rcc.c:775
   2:	4a05      	ldr	r2, [pc, #20]	(18 <RCC_AHBPeriphClockCmd+0x18>)
   4:	6953      	ldr	r3, [r2, #20]
   6:	ea40 0303 	orr.w	r3, r0, r3
   a:	e003      	b.n	14 <RCC_AHBPeriphClockCmd+0x14>
D:\STM32\Program\1.11_Odchudzanie\um0427\FWLib\library\src/stm32f10x_rcc.c:779
   c:	4a02      	ldr	r2, [pc, #8]	(18 <RCC_AHBPeriphClockCmd+0x18>)
   e:	6953      	ldr	r3, [r2, #20]
  10:	ea23 0300 	bic.w	r3, r3, r0
  14:	6153      	str	r3, [r2, #20]
D:\STM32\Program\1.11_Odchudzanie\um0427\FWLib\library\src/stm32f10x_rcc.c:781
  16:	4770      	bx	lr
  18:	40021000 	.word	0x40021000
Disassembly of section .text.RCC_APB2PeriphClockCmd:

00000000 <RCC_APB2PeriphClockCmd>:
RCC_APB2PeriphClockCmd():
D:\STM32\Program\1.11_Odchudzanie\um0427\FWLib\library\src/stm32f10x_rcc.c:806
   0:	b121      	cbz	r1, c <RCC_APB2PeriphClockCmd+0xc>
D:\STM32\Program\1.11_Odchudzanie\um0427\FWLib\library\src/stm32f10x_rcc.c:808
   2:	4a05      	ldr	r2, [pc, #20]	(18 <RCC_APB2PeriphClockCmd+0x18>)
   4:	6993      	ldr	r3, [r2, #24]
   6:	ea40 0303 	orr.w	r3, r0, r3
   a:	e003      	b.n	14 <RCC_APB2PeriphClockCmd+0x14>
D:\STM32\Program\1.11_Odchudzanie\um0427\FWLib\library\src/stm32f10x_rcc.c:812
   c:	4a02      	ldr	r2, [pc, #8]	(18 <RCC_APB2PeriphClockCmd+0x18>)
   e:	6993      	ldr	r3, [r2, #24]
  10:	ea23 0300 	bic.w	r3, r3, r0
  14:	6193      	str	r3, [r2, #24]
D:\STM32\Program\1.11_Odchudzanie\um0427\FWLib\library\src/stm32f10x_rcc.c:814
  16:	4770      	bx	lr
  18:	40021000 	.word	0x40021000
Disassembly of section .text.RCC_APB1PeriphClockCmd:

00000000 <RCC_APB1PeriphClockCmd>:
RCC_APB1PeriphClockCmd():
D:\STM32\Program\1.11_Odchudzanie\um0427\FWLib\library\src/stm32f10x_rcc.c:840
   0:	b121      	cbz	r1, c <RCC_APB1PeriphClockCmd+0xc>
D:\STM32\Program\1.11_Odchudzanie\um0427\FWLib\library\src/stm32f10x_rcc.c:842
   2:	4a05      	ldr	r2, [pc, #20]	(18 <RCC_APB1PeriphClockCmd+0x18>)
   4:	69d3      	ldr	r3, [r2, #28]
   6:	ea40 0303 	orr.w	r3, r0, r3
   a:	e003      	b.n	14 <RCC_APB1PeriphClockCmd+0x14>
D:\STM32\Program\1.11_Odchudzanie\um0427\FWLib\library\src/stm32f10x_rcc.c:846
   c:	4a02      	ldr	r2, [pc, #8]	(18 <RCC_APB1PeriphClockCmd+0x18>)
   e:	69d3      	ldr	r3, [r2, #28]
  10:	ea23 0300 	bic.w	r3, r3, r0
  14:	61d3      	str	r3, [r2, #28]
D:\STM32\Program\1.11_Odchudzanie\um0427\FWLib\library\src/stm32f10x_rcc.c:848
  16:	4770      	bx	lr
  18:	40021000 	.word	0x40021000
Disassembly of section .text.RCC_APB2PeriphResetCmd:

00000000 <RCC_APB2PeriphResetCmd>:
RCC_APB2PeriphResetCmd():
D:\STM32\Program\1.11_Odchudzanie\um0427\FWLib\library\src/stm32f10x_rcc.c:872
   0:	b121      	cbz	r1, c <RCC_APB2PeriphResetCmd+0xc>
D:\STM32\Program\1.11_Odchudzanie\um0427\FWLib\library\src/stm32f10x_rcc.c:874
   2:	4a05      	ldr	r2, [pc, #20]	(18 <RCC_APB2PeriphResetCmd+0x18>)
   4:	68d3      	ldr	r3, [r2, #12]
   6:	ea40 0303 	orr.w	r3, r0, r3
   a:	e003      	b.n	14 <RCC_APB2PeriphResetCmd+0x14>
D:\STM32\Program\1.11_Odchudzanie\um0427\FWLib\library\src/stm32f10x_rcc.c:878
   c:	4a02      	ldr	r2, [pc, #8]	(18 <RCC_APB2PeriphResetCmd+0x18>)
   e:	68d3      	ldr	r3, [r2, #12]
  10:	ea23 0300 	bic.w	r3, r3, r0
  14:	60d3      	str	r3, [r2, #12]
D:\STM32\Program\1.11_Odchudzanie\um0427\FWLib\library\src/stm32f10x_rcc.c:880
  16:	4770      	bx	lr
  18:	40021000 	.word	0x40021000
Disassembly of section .text.RCC_APB1PeriphResetCmd:

00000000 <RCC_APB1PeriphResetCmd>:
RCC_APB1PeriphResetCmd():
D:\STM32\Program\1.11_Odchudzanie\um0427\FWLib\library\src/stm32f10x_rcc.c:905
   0:	b121      	cbz	r1, c <RCC_APB1PeriphResetCmd+0xc>
D:\STM32\Program\1.11_Odchudzanie\um0427\FWLib\library\src/stm32f10x_rcc.c:907
   2:	4a05      	ldr	r2, [pc, #20]	(18 <RCC_APB1PeriphResetCmd+0x18>)
   4:	6913      	ldr	r3, [r2, #16]
   6:	ea40 0303 	orr.w	r3, r0, r3
   a:	e003      	b.n	14 <RCC_APB1PeriphResetCmd+0x14>
D:\STM32\Program\1.11_Odchudzanie\um0427\FWLib\library\src/stm32f10x_rcc.c:911
   c:	4a02      	ldr	r2, [pc, #8]	(18 <RCC_APB1PeriphResetCmd+0x18>)
   e:	6913      	ldr	r3, [r2, #16]
  10:	ea23 0300 	bic.w	r3, r3, r0
  14:	6113      	str	r3, [r2, #16]
D:\STM32\Program\1.11_Odchudzanie\um0427\FWLib\library\src/stm32f10x_rcc.c:913
  16:	4770      	bx	lr
  18:	40021000 	.word	0x40021000
Disassembly of section .text.RCC_BackupResetCmd:

00000000 <RCC_BackupResetCmd>:
RCC_BackupResetCmd():
D:\STM32\Program\1.11_Odchudzanie\um0427\FWLib\library\src/stm32f10x_rcc.c:928
   0:	4b01      	ldr	r3, [pc, #4]	(8 <RCC_BackupResetCmd+0x8>)
   2:	6018      	str	r0, [r3, #0]
D:\STM32\Program\1.11_Odchudzanie\um0427\FWLib\library\src/stm32f10x_rcc.c:929
   4:	4770      	bx	lr
   6:	46c0      	nop			(mov r8, r8)
   8:	42420440 	.word	0x42420440
Disassembly of section .text.RCC_ClockSecuritySystemCmd:

00000000 <RCC_ClockSecuritySystemCmd>:
RCC_ClockSecuritySystemCmd():
D:\STM32\Program\1.11_Odchudzanie\um0427\FWLib\library\src/stm32f10x_rcc.c:944
   0:	4b01      	ldr	r3, [pc, #4]	(8 <RCC_ClockSecuritySystemCmd+0x8>)
   2:	6018      	str	r0, [r3, #0]
D:\STM32\Program\1.11_Odchudzanie\um0427\FWLib\library\src/stm32f10x_rcc.c:945
   4:	4770      	bx	lr
   6:	46c0      	nop			(mov r8, r8)
   8:	4242004c 	.word	0x4242004c
Disassembly of section .text.RCC_MCOConfig:

00000000 <RCC_MCOConfig>:
RCC_MCOConfig():
D:\STM32\Program\1.11_Odchudzanie\um0427\FWLib\library\src/stm32f10x_rcc.c:966
   0:	4b01      	ldr	r3, [pc, #4]	(8 <RCC_MCOConfig+0x8>)
   2:	7018      	strb	r0, [r3, #0]
D:\STM32\Program\1.11_Odchudzanie\um0427\FWLib\library\src/stm32f10x_rcc.c:967
   4:	4770      	bx	lr
   6:	46c0      	nop			(mov r8, r8)
   8:	40021007 	.word	0x40021007
Disassembly of section .text.RCC_GetFlagStatus:

00000000 <RCC_GetFlagStatus>:
RCC_GetFlagStatus():
D:\STM32\Program\1.11_Odchudzanie\um0427\FWLib\library\src/stm32f10x_rcc.c:989
   0:	0943      	lsrs	r3, r0, #5
D:\STM32\Program\1.11_Odchudzanie\um0427\FWLib\library\src/stm32f10x_rcc.c:1000
   2:	2b01      	cmp	r3, #1
D:\STM32\Program\1.11_Odchudzanie\um0427\FWLib\library\src/stm32f10x_rcc.c:989
   4:	d102      	bne.n	c <RCC_GetFlagStatus+0xc>
D:\STM32\Program\1.11_Odchudzanie\um0427\FWLib\library\src/stm32f10x_rcc.c:1002
   6:	4b08      	ldr	r3, [pc, #32]	(28 <RCC_GetFlagStatus+0x28>)
   8:	681b      	ldr	r3, [r3, #0]
   a:	e005      	b.n	18 <RCC_GetFlagStatus+0x18>
D:\STM32\Program\1.11_Odchudzanie\um0427\FWLib\library\src/stm32f10x_rcc.c:1004
   c:	2b02      	cmp	r3, #2
D:\STM32\Program\1.11_Odchudzanie\um0427\FWLib\library\src/stm32f10x_rcc.c:1006
   e:	bf0b      	itete	eq
  10:	4b05      	ldreq	r3, [pc, #20]	(28 <RCC_GetFlagStatus+0x28>)
D:\STM32\Program\1.11_Odchudzanie\um0427\FWLib\library\src/stm32f10x_rcc.c:1010
  12:	4b05      	ldrne	r3, [pc, #20]	(28 <RCC_GetFlagStatus+0x28>)
D:\STM32\Program\1.11_Odchudzanie\um0427\FWLib\library\src/stm32f10x_rcc.c:1006
  14:	6a1b      	ldreq	r3, [r3, #32]
D:\STM32\Program\1.11_Odchudzanie\um0427\FWLib\library\src/stm32f10x_rcc.c:1010
  16:	6a5b      	ldrne	r3, [r3, #36]
  18:	f000 001f 	and.w	r0, r0, #31	; 0x1f
  1c:	fa33 f000 	lsrs.w	r0, r3, r0
D:\STM32\Program\1.11_Odchudzanie\um0427\FWLib\library\src/stm32f10x_rcc.c:1027
  20:	f000 0001 	and.w	r0, r0, #1	; 0x1
  24:	4770      	bx	lr
  26:	46c0      	nop			(mov r8, r8)
  28:	40021000 	.word	0x40021000
Disassembly of section .text.RCC_WaitForHSEStartUp:

00000000 <RCC_WaitForHSEStartUp>:
RCC_WaitForHSEStartUp():
D:\STM32\Program\1.11_Odchudzanie\um0427\FWLib\library\src/stm32f10x_rcc.c:200
   0:	b510      	push	{r4, lr}
D:\STM32\Program\1.11_Odchudzanie\um0427\FWLib\library\src/stm32f10x_rcc.c:206
   2:	2031      	movs	r0, #49
   4:	f7ff fffe 	bl	0 <RCC_WaitForHSEStartUp>
   8:	4a09      	ldr	r2, [pc, #36]	(30 <RCC_WaitForHSEStartUp+0x30>)
   a:	7010      	strb	r0, [r2, #0]
D:\STM32\Program\1.11_Odchudzanie\um0427\FWLib\library\src/stm32f10x_rcc.c:207
   c:	6853      	ldr	r3, [r2, #4]
   e:	3301      	adds	r3, #1
  10:	6053      	str	r3, [r2, #4]
D:\STM32\Program\1.11_Odchudzanie\um0427\FWLib\library\src/stm32f10x_rcc.c:208
  12:	7813      	ldrb	r3, [r2, #0]
  14:	b923      	cbnz	r3, 20 <RCC_WaitForHSEStartUp+0x20>
  16:	6852      	ldr	r2, [r2, #4]
  18:	f240 13ff 	movw	r3, #511	; 0x1ff
  1c:	429a      	cmp	r2, r3
  1e:	d1f0      	bne.n	2 <RCC_WaitForHSEStartUp+0x2>
D:\STM32\Program\1.11_Odchudzanie\um0427\FWLib\library\src/stm32f10x_rcc.c:211
  20:	2031      	movs	r0, #49
  22:	f7ff fffe 	bl	0 <RCC_WaitForHSEStartUp>
D:\STM32\Program\1.11_Odchudzanie\um0427\FWLib\library\src/stm32f10x_rcc.c:221
  26:	3800      	subs	r0, #0
  28:	bf18      	it	ne
  2a:	2001      	movne	r0, #1
  2c:	bd10      	pop	{r4, pc}
  2e:	46c0      	nop			(mov r8, r8)
  30:	00000000 	.word	0x00000000
Disassembly of section .text.RCC_ClearFlag:

00000000 <RCC_ClearFlag>:
RCC_ClearFlag():
D:\STM32\Program\1.11_Odchudzanie\um0427\FWLib\library\src/stm32f10x_rcc.c:1040
   0:	4a02      	ldr	r2, [pc, #8]	(c <RCC_ClearFlag+0xc>)
   2:	6a53      	ldr	r3, [r2, #36]
   4:	f043 7380 	orr.w	r3, r3, #16777216	; 0x1000000
   8:	6253      	str	r3, [r2, #36]
D:\STM32\Program\1.11_Odchudzanie\um0427\FWLib\library\src/stm32f10x_rcc.c:1043
   a:	4770      	bx	lr
   c:	40021000 	.word	0x40021000
Disassembly of section .text.RCC_GetITStatus:

00000000 <RCC_GetITStatus>:
RCC_GetITStatus():
D:\STM32\Program\1.11_Odchudzanie\um0427\FWLib\library\src/stm32f10x_rcc.c:1060
   0:	4b03      	ldr	r3, [pc, #12]	(10 <RCC_GetITStatus+0x10>)
   2:	689b      	ldr	r3, [r3, #8]
   4:	4218      	tst	r0, r3
D:\STM32\Program\1.11_Odchudzanie\um0427\FWLib\library\src/stm32f10x_rcc.c:1078
   6:	bf0c      	ite	eq
   8:	2000      	moveq	r0, #0
   a:	2001      	movne	r0, #1
   c:	4770      	bx	lr
   e:	46c0      	nop			(mov r8, r8)
  10:	40021000 	.word	0x40021000
Disassembly of section .text.RCC_ClearITPendingBit:

00000000 <RCC_ClearITPendingBit>:
RCC_ClearITPendingBit():
D:\STM32\Program\1.11_Odchudzanie\um0427\FWLib\library\src/stm32f10x_rcc.c:1095
   0:	4b01      	ldr	r3, [pc, #4]	(8 <RCC_ClearITPendingBit+0x8>)
   2:	7018      	strb	r0, [r3, #0]
D:\STM32\Program\1.11_Odchudzanie\um0427\FWLib\library\src/stm32f10x_rcc.c:1102
   4:	4770      	bx	lr
   6:	46c0      	nop			(mov r8, r8)
   8:	4002100a 	.word	0x4002100a
